:0894090033302E312020200039
:107F4600C10DC109C10CC10E4113A2004213A0000C
:107F5600004113A4014113670144136DFFFFFFFFA6
:027F6600C10B4D
:10694000EFFD3395E0FC746D2DF58274133CF583F7
:10695000222582F582E43583F5837401F09013CF0C
:10696000E475F001024A0B9011C9124D1689828A12
:106970008322EEFD3395E0FC74682DF58274133CA0
:10698000F58322900939E0D36480F8EE6480982280
:106990009013D0E025E0FF9013CFE033FE74162F64
:1069A000F58274053EF583229013CFE0FEA3E0FF4D
:1069B000229013EA124D369000051248EBFF90002A
:1069C000061248EBFD9000040248EBE49013CFF070
:1069D000A3F0227B017A1379D79013EA124D3690F7
:1069E00000031248EBFF90139FE06F22EDFF3395F9
:1069F000E0FEEF25E0FFEE33FE2274FC2FF58274FB
:106A0000053EF58322FBEAC4F854F0C8EBC4540FEA
:106A100048901515F0229013CFE0FCA3E02224DE6D
:106A2000F58274053EF583E02212922A90093CE03B
:106A3000223EF583EAF0A3EBF0223EF583E0FAA3D1
:106A4000E02225E02480F582E43405F58322EC255C
:106A5000E02425F8E6FA08E6229FEE6480F8E06478
:036A6000809822F9
:10926F0075840F75A4357580C075A57C75A7FF75BE
:06927F00E11775E3442233
:0F933D00E4F584759A4075F809759D01C2FA220E
:108E0700E4F584758850758921F58E758DEB75C9E4
:108E17000875CDFF75CCC075CBFF75CAE075C80462
:038E2700F58422AD
:1092EA00E4F584759105759852758401F598F584AD
:0192FA002251
:1085AB00E4FFFE75840F438A0353A1DFF58475B78F
:1085BB003075840F43A120438901758D01758F019F
:1085CB00758E040FBF00010EEF640F4E70F54389DB
:1085DB0002E58920E4130FBF00010EBE0FF3BFFFAE
:0C85EB00F0E4F58443EF1080E87597027F
:0185F7002261
:0A93E20075A89275B81075E6082210
:1092D800E4F58475D84075D98375DA3175DB31D2F8
:0292E800DE2284
:10929B0012926F1285AB128E071292D81292EA12AB
:0592AB00933D0293E277
:1092B0007F021291127F041291127F0212922A7F72
:0492C0000402922AE8
:02712C00AC07AE
:10712E00E4901516F0ED4430901514F0E4FD746102
:10713E002DF8E66C705790151604F01269EC7495E4
:10714E002FF5827402126A3A126A05EB540FF91285
:10715E0069EC74D92FF5827401126A3AFB74952F7B
:10716E00F5827402126A3174F02FF5827400126A7D
:10717E003AFB74D92FF5827401126A31126A4EFBF2
:10718E001269EC74F02FF5827400126A310DED6401
:10719E0004709B901516E0700C126A4E126A05AFC1
:1071AE0003EF540FF9E9C454F0F9E59A20E7FBE434
:1071BE00F59BE59A20E7FB901514E0F59BE59A20E8
:1071CE00E7FB901515E0F59BE59A20E7FB899BE51B
:0B71DE009A20E7FBAF05EF3395E0FEC1
:0171E9002283
:0575E400901523EFF0FB
:1075E900124D6B760800761501762202762F037606
:1075F9003C047649057656067663070000766E7F69
:10760900061264669015247405F080597F06125B92
:10761900DB9015247406F0804C7F06127A9C901535
:10762900247407F0803F7F0612706990152474084E
:10763900F080327F071264669015247409F0802562
:107649007F07125BDB901524740AF080187F0712FC
:107659007A9C901524740BF0800B7F071270699047
:107669001524740CF0D282C295901524E0FF901570
:0A76790023E0FD12712CD295C282AD
:0176830022E4
:05768400901525EFF058
:10768900124D6B76A80076B50176C20276CF0376E5
:10769900DC0476E90576F6067703070000770E7FA6
:1076A90008126466901526740DF080597F08125BE4
:1076B900DB9015267412F0804C7F08127A9C901585
:1076C90026740FF0803F7F08127069901526741098
:1076D900F080327F091264669015267411F08025B6
:1076E9007F09125BDB901526740EF080187F091252
:1076F9007A9C9015267413F0800B7F09127069909B
:1077090015267414F0D282C296901526E0FF9015C2
:0A77190025E0FD12712CD296C28209
:017723002243
:05846600901527EFF066
:10846B0024FA601704702B901528741DF0901413C8
:10847B007403F07B277D2A7F1D8012901528741CB6
:10848B00F09014137402F07B117D1F7F1C126C94FF
:10849B00800A901527E0FFA3F0125960D282C29494
:1084AB00901528E0FF901527E0FD12712CD294C295
:0184BB00823E
:0184BC00229D
:0583B600901529EFF015
:1083BB0024FA601704702A90152A741BF09014137A
:1083CB007401F07B287D2B7F1B801190152A741A6A
:1083DB00F0E4901413F07B127D207F1A126C9480C2
:1083EB000C901529E02415FFA3F0127724D282C23A
:1083FB009790152AE0FF901529E0FD12712CD2976A
:02840B00C2822B
:01840D00224C
:0F934C009013667407F0D294D295D296D29722DE
:106EA40090152BE584F0A3E5A8F09011B0124D16CF
:106EB400E94A7003026FA153A87DE4F58453F87F77
:106EC4009013A5F0A3F0C2B3901266E0FFB40118CA
:106ED40090119AE0C313FE7402A806088002C3331B
:106EE400D8FC9013A5F0806CEFB40216901238E031
:106EF400FF7401A807088002C333D8FC9013A6F0DE
:106F04008052901266E0B4034B90119FE0124D6BD7
:106F14006F36006F36016F3E026F3E036F46046F9B
:106F240046056F4E066F4E076F56086F56090000F0
:106F34006F589013A67410F0801A9013A67420F062
:106F440080129013A67440F0800A9013A67480F007
:106F54008002D2B3300A079013A5E04440F0C2FA8D
:106F6400E4FF0FEFB432FB53F87FE59A20E7FB9080
:106F740013A5E0F59BE4FF0FEFB432FB53F87FE574
:106F84009A20E7FB9013A6E0F59BE4FF0FEFB432E1
:0D6F9400FBD2FA90152BE0F584A3E0F5A8E0
:016FA10022CD
:035006000273F939
:1073F900C0E0C0F0C083C082C0D075D000C000C05A
:0D74090001C002C003C004C005C006C007DA
:107416009013A0126960901366E014F0E0C394071D
:1074260050037426F0901366E0FF131313541FFEE7
:10743600EF5407901543F0AF06EF24FE6018146072
:107446001F1460262403702E901543E0FF64076026
:10745600251284668020901543E0FF1275E480169D
:10746600901543E0FF127684800C901543E0FF648C
:0C7476000760031283B6758AFF758CFF57
:10748200D007D006D005D004D003D002D001D0005E
:0B749200D0D0D082D083D0F0D0E03208
:0A93EC00EF126A42ECF0A3EDF0224C
:10810F00E4FE1269835011EE126941E0F460061229
:10811F006978E004F00E80EA901371E0126941EF84
:10812F00F0126978E4F0FE1269835011EE12694182
:10813F00E0B4FF06901371EEF0220E80EAE4901384
:10814F0071F0901368E0FF7E01126983501A126973
:10815F0072E0FDD3EF6480F8ED6480984007AF05BF
:08816F00901371EEF00E80E1A7
:0181770022E5
:0571EA0090152DEFF0EF
:1071EF00E4FF900939E0D36480F8EF648098506B26
:1071FF00126940E0FE90152DE0FDEE6D7059126999
:10720F004074FFF012697874FFF090152E747FF0C0
:10721F00E4FE126983501CEE6F6015126972E0FD77
:10722F0090152EE0C36480F8ED6480985002EDF065
:10723F000E80DFE4FE1269835021EE6F6016126933
:10724F0072C083C082E0FD90152EE0FCC3ED9CD090
:10725F0082D083F00E80DE0F0271F1E4901371F093
:10726F00FF900939E0FED36480F8EF6480985010E6
:10727F00126940E0F4601A901371E004F00F80E19E
:10728F00EE14FF901371E0FED3EF1269884002EF06
:01729F00F0FE
:0172A00022CB
:109112007584014398028F99E59870047F0180025B
:0A9122007F00EF20E1F2E4F5842263
:10922A00E4F5844398028F99E59870047F018002DF
:07923A007F00EF20E1F222AA
:02830200A907C9
:10830400E490152FF0A3F0E9FF3395E0FEC3901538
:1083140030E090152F126A59503EE4FFFEE9FD3318
:1083240095E0FCC3EF9DEC1269885024E4FDFCE960
:10833400FB3395E0FAC3ED9BEA6480F8EC64809823
:1083440050070DBD00010C80E60FBF00010E80CD6B
:0883540090152F12696080AF43
:01835C0022FE
:10409A00E4900939F0FBFAF99011B0124D3675FF28
:1040AA00DE75FFADE4F5E6F5E7128FB812929B12C2
:1040BA00914612934C128E9212930CE4F58475D4A5
:1040CA008475D48475D10375D340D281128BB3D24F
:1040DA00AFD2FF1269CB90139F7440F0FF1293780E
:1040EA0043F602E4901371F01269CC900939E0FFAB
:1040FA003395E0FED39013D0E09013CF126A595053
:10410A0022E0FEA3E0FF246DF58274133EF583746A
:10411A00FFF074682FF58274133EF58374FF1269F9
:10412A005C80C8E41247D1127BBA128FF512940050
:10413A00126EA47F3912922AC2091291947E00EF5C
:10414A00640160030245B5128DBEEF64B0600302DC
:10415A0045B59013D6F01269CC1269A8C3942DEE16
:10416A0064809480501474722FF58274133EF58320
:10417A00E4F09013CF12696180DF1269CB1269A84B
:10418A00C3941BEE648094805028126A16FD24FCA6
:10419A00F58274053CF583E0FB74DE2DF582740527
:1041AA003CF583EBF01269FAE4F09013CF126961DF
:1041BA0080CBC219129194EF60FA128DBE9013D17E
:1041CA00EFF05480FFE4FCFDFEEF700302432DE0A4
:1041DA00FF64C0700302432DEF64B0700302432DE5
:1041EA009013D6E004F09013D1E0547FFFA3F0744B
:1041FA0019D39F500DE0FF94265007EF24F2A3F045
:10420A00802A9013D2E0FFE4D39F500AEF9418500B
:10421A0005A3EFF08016EFB429089013D37419F0B0
:10422A00800AEFB42C069013D3741AF09013D3E0DB
:10423A00FFC3941B500D74FC2FF582E43405F583FB
:10424A007401F0E49013D4F0A3F0129194EF60FAA1
:10425A00128DBEAD07129194EF60FA128DBEAC07B3
:10426A00AF059013D4E0F0A3E04FF09013D4E0FE32
:10427A00A3E07806C333CE33CED8F9F0EE9013D448
:10428A00F0AF04E0F0A3E04FF09013D2E0126A42DC
:10429A00E0FEA3E04E705E1269CC1269A8C39405D1
:1042AA00EE64809480501FEF75F02DA424F8F582F7
:1042BA00E43400F583C083C0829013D2E0D082D068
:1042CA008312695180D41269CB1269A8C39404EE8F
:1042DA0064809480501FEF75F02DA424E1F582E4E8
:1042EA003401F583C083C0829013D2E0D082D08398
:1042FA0012695180D49013D2E0FF9013D4E0FCA34A
:10430A00E0FD1293EC9013D2E0FF2472F582E434BC
:10431A0013F5837401F090136CEFF0201905128DD8
:10432A00E3D2199013D1E064C060030241BE901237
:10433A0037E060081282A1300D02C20D1269CB1259
:10434A0069A8C3941BEE6480948040030244D87425
:10435A00DE2F126A20600302448A9013CFA3E0245E
:0C436A00FC1269FDE06401600302448A5B
:104376009013F0F0A3F09013F0E0FEA3E0FFC394D7
:1043860004EE64809480504C90074575F07DEF12E2
:104396004CF1EE75F07DA42583F583C083C08212AF
:1043A60069A8D082D08375F005124CF1EE75F00540
:1043B600A42583F583E0540F60129013F0E0FCA36C
:1043C600E024DAF58274053CF583EFF09013F012E1
:1043D600696080A29013CFA3E0FF12810F126A16C4
:1043E600FD25E0FFEC12699B7414F0A3E4F07496CB
:1043F6002FF58274003EF583C083C082E04410FF2F
:10440600A3E0D082D083CFF0A3EFF0901237E07014
:10441600030244D2ED64124C60047F0180027F00E7
:10442600126A16FD64114C60047E0180027E00EE65
:104436005F70030244D2D20D9011AD124D168D82DB
:104446008C837405124CE01248EB540F70047F0104
:1044560080027F00EF540FFF9011AD124D16126AC5
:1044660016F5828C837405124CE0E92582F9EA354B
:1044760083FA1248D254F04F12493A12500312945A
:014486000035
:104487000244D21269A8126A1EB4010B1269FAE03B
:1044970070051271EA80341269A8126A1E640170ED
:1044A7002A1269FAE0B40123126990E0FCA3E0D371
:1044B7009400EC9402400D12699D74FE75F0001291
:1044C7004A0B8007126990E4F0A3F012695D02437A
:1044D700491269CBFDFC900615E0FF601C9005F7BB
:1044E700E070160D90093BE090136760057401F0CA
:1044F7008007E0FEC374019EF0EF70159005F7E0AA
:10450700600F7C007D0190093BE06005E490136734
:10451700F0900616E0FF60229005F8E0701C9013FB
:10452700CFF0A304F090093AE09013A4600574015A
:10453700F08007E0FEC374019EF0EF70199005F854
:10454700E060139013CFE4F0A304F090093AE06021
:1045570005E49013A4F09013CFE07002A3E0602568
:104567009013A4E0600F7F02126A2960047F048021
:10457700117F02800D7F01126A2960047F03800288
:104587007F01129112ED4C6025901367E0600F7F59
:1045970004126A2960047F0280117F04800D7F0363
:1045A700126A2960047F0180027F03129112128C24
:1045B7008FEF700302466512850FEF124D6B463081
:1045C70001462502463B0445F10545EA0645FF0736
:1045D70045F808460D0946060A461B0B46140C000B
:1045E70000464F1269677FFF802F1269677F01803E
:1045F700281269677FFE80211269677F02801A127D
:1046070069677FFD80131269677F03800C126967F2
:104617007FFC80051269677F04124D9580279012F1
:104627006B124D16124D91801C9011CC124D161223
:104637004D918011300B04B20A800AE49006CBF04A
:10464700129212C20A126EA4128C8FEF60030245F7
:10465700BE9013A07427F0A37410F0129400300CCE
:104667001090139FE0FF7BFF7A94790912840EC2A2
:104677000C300E0A90139FE0FF1291AEC20E7B0121
:104687007A1379D7128E70EF70030241429013D9D3
:10469700E0124D6B46FC04470D0546C61446BA1694
:1046A70046BE1746CB1A46E51B46F01D46F61E00CA
:1046B70000472AD20A8002C20A126EA402472AD2EF
:1046C7000B02472A7B017A1379D79013E7124D36ED
:1046D7001248D2FE90139FE0FF6E7047800590133B
:1046E7009FE0FF12924102472A12941902472A12A9
:1046F700946502472A1269D37029300A1E1269B1DC
:10470700FB1280A380151269D37018300A0D126945
:10471700B1FB127DCB128D9912940090139FE0FF8D
:104727001291C7200A030246859013D9E014601A34
:1047370024FA602114604C24066003024685124760
:10474700A49006CBF012921280331247A41247D1DD
:1047570012940080281247BA1269C5FD900005120D
:1047670048EBFBC0039013ED124D1690000612485C
:10477700EB90143FF0D0031278531294001293B6C3
:104787000246851247BA1269C5FD9000051248EB2B
:0D479700FB126A631294001293B60246856D
:1047A4001292FB7B017A1379D79013E7124D36905E
:1047B40000031248EB221292FB7B017A1379D79003
:1047C40013ED124D369000031248EBFF229006CBF6
:0847D400F0128D991292B0223F
:10912C007B01E49014B9F0227422F0A3EFF0A32297
:0A913C007B01E49014B9F07D0422D9
:0B8905009014B5124D369014B8EDF040
:10891000E49014BAF09014B5124D169014B8E0908B
:1089200014A4F09014B9E09014A5F0E4FF12803480
:10893000EFB4FF0D9014BAE0FE04F0EEC3940340D0
:03894000D47E00E2
:018943002211
:068E7000901517124D36AB
:108E76007E007F007D10124DC4901517124D167D91
:0B8E86001012749DEF7002FF227F01AC
:018E910022BE
:10840E0090145E1291347413F01248D2901461F0ED
:10841E009000011248EB901462F09000021248EBAB
:10842E00901463F09000031248EB901464F09000E7
:10843E00041248EB901465F09000051248EB90146E
:10844E0066F09000061248EB901467F07A14795E8D
:08845E0012912C7D0A02890530
:1091AE009014E81291347403F0A374FFF07A1479DA
:0991BE00E812912C7D04028905E0
:109241009014EC129134741CF0A374FFF07A147929
:07925100EC12913C028905BB
:1091C700E49014F0F0A3EFF0A3740AF0A3EFF07AA1
:0991D7001479F012913C028905A3
:108D2A00E0FEA3E0A60608F6E4F584C2AF43B70165
:108D3A0022E475F001124A2185F082F58322EEF0D1
:058D4A00A3EFF0A322DD
:108AA800AB84A2AF921AE4FCFDED9014F4124CA32F
:108AB8009014F6781D128D2A438F02438F0118E611
:108AC800FE08E6F5828E83E4F053B7FEF58FA21A0E
:068AD80092AFAF038F8492
:018ADE002275
:02888100AB0545
:10888300AA84A2AF921BE4FCFDED9014F8124CA352
:10889300EBFF3395E0FEEFF44E601C9014FA78780A
:1088A300128D2A758F0118E6FC08E6F5828C83EB9E
:0F88B300F053B7FEE4F58FA21B92AFAF028F8494
:0188C2002293
:1084BD009014BB128D48ECF0A3EDF0A3EAF0A3EB02
:1084CD00F09014BFE07002A3E060369014BBE0FEA4
:1084DD00A3E0FFA3E0FCA3E0F5828C83E0FD12880E
:1084ED00819014BF74FFF5F0124A0B9014BDE47522
:1084FD00F001124A0B9014BBE475F001124A0B8087
:02850D00C0228A
:08941100E4900BAEF0A3F02281
:108D0400900BAEE0FEA3E0FF128AA8900BAEE0FE4B
:108D1400A3E0FF7C0B7DB07B007A041284BDE49059
:068D24000BAEF0A3F022EB
:0A7FBD00A9059014C1EEF0A3EFF047
:107FC700EE54FCFE900BAEE0FCA3E0FD7002EE6CFD
:107FD7006042ED4C6003128D049014C1E0FEEE5434
:107FE700FCFE7F00900BAEF0A3EFF09014C3128D50
:107FF70048740BF0A374B0F07E049014C3128D3B49
:10800700E493FD9014C5128D3BEDF0EF1F70011E38
:10801700EF4E70E69014C1E0FCA3E0FDEC5403FCC6
:0C80270074B02DF582740B3CF583E9F079
:01803300222A
:108A7000901499128D48124D3690149E74FFF5F0A3
:108A8000124A2145F06020901499E475F001124AD1
:108A900021AFF0FE90149BE475F001124D1F1248B7
:088AA000D2FD127FBD80D2223D
:107F6800421364000042130F000042130A0000C1CC
:057F780011C110C10F52
:1089FC00901305E475F001024A0BD3901365E094D3
:108A0C0000901364E06480948022E0FEA3E02411C3
:108A1C00F58274132290130AF0A3F02274FFF5F080
:0A8A2C00024A0BFCE5F064404C2206
:0A93F600C210C211E490130EF02221
:108F1900E4901364F0A3F090130FF0A3F0A3F01200
:108F29008A21901305F0A37440F0E490130DF02208
:065009001293F6028F195C
:1091E000E4F5848FC343C30175C04475CF8EC2C3F9
:0991F00043E60290130C04F02286
:1092FB00E4F58420C7FDC2C2125009E490130CF0B0
:01930B00223F
:0B93B600E4F584D2C290130C04F022F6
:0D937800AE071291E0901309EFF0025009CA
:108D4F00E4901531F0A3F0301002FF222011FDD274
:108D5F0010901307E4F0A37410F0901352EFF0E4A7
:048D6F00A3F07F01ED
:018D730022DD
:108BE30030100A901307E07002A3E070037F0022A5
:108BF300901307128A28901353E0FE04F074542E46
:0C8C0300F582E43413F583EFF07F0122CA
:0B93C100301007C210D21112935B2283
:0E935B00AF84E4F58420C7FDC2C4D2C58F8460
:0193690022E1
:108034009014A1124D3690130CE07002FF2290149C
:10804400A4E0FE6005D3941040037F0022128D4FFC
:03805400EF604991
:10805700E49014A6F09014A4E0FF9014A6E0FEC3E9
:108067009F501F9014A1124D168E827583001248DF
:10807700EBFF128BE3EF7002FF229014A6E004F0EF
:1080870080D3E490130EF01293C19014A5E070030F
:098097002011FD90130EE0FF2200
:0380A0007FFF223D
:0B749D009014FC124D369014FFEDF02F
:1074A800E4FF128A0650012253E6FD90130A128A5D
:1074B800163EF583E0FF90130A1289FF128A2F7097
:1074C80003128A211289FCE4FE9014FFE0FDEEC34A
:1074D8009D5035EEC39F503090130AE0FC128A1875
:1074E8003CF583E0FD9014FC124D168E82758300E6
:1074F800ED12494C90130A1289FF128A2F70031259
:107508008A211289FC0E80C1EEC39F501490130A81
:107518001289FF128A2F7003128A211289FC0E80A9
:10752800E7901364128A2843E6029014FFE0FEEF06
:08753800C39E50028002AF0661
:017540002228
:0C939200128A0640047F0180027F002246
:035018000265AF7F
:1065AF00C0E0C0F0C083C082C0D075D000C000C0B2
:0365BF0006C0070C
:1065C200C21CAFC1EF124D6B65F80865F810660882
:1065D20018660D20661A28664730665238665A6079
:1065E200665568665A70665578666180666190661F
:1065F200BDA0000066CB901352E0F5C2C2C5901355
:1066020051E4F00266CD901353802890130E74FD6E
:10661200F0D2C4D2C50266CD901353E0FF9013515D
:10662200E0C39F5014E0FF04F074542FF582E43469
:1066320013F583E0F5C20266CDD2C490130EE4F0E6
:10664200C2110266CDD2C590130E74FEF00266CD61
:106652000266C2D20F0266CD901304E4F0806C9001
:106662001304E07020E5C2F0E0FFC3901306E09F40
:106672007480F8901305E06480985003128F19908B
:106682001304E004F0901305128A2890130F128A63
:10669200163EF583E5C2F090130F1289FFFEE5F076
:1066A20064404E700690130FF0A3F0901304E014B0
:1066B200F07018901364128A008010300F0DC20F10
:1066C200901351E4F0D2C58002D21C301C0EC2C617
:0E66D200D2C6C2C5C2C4D2C2C21CC211C2C34B
:1066E000D007D006D000D0D0D082D083D0F0D0E078
:0166F0003277
:05501200A2C7E433FF1A
:015017002276
:10931D000001FF00FF000001010000FF00FF010040
:108ADF00E56785688385698222901501024D16D35B
:108AEF00ED9408EC6480948022D3ED9410EC6480B4
:108AFF00948022C3ED94F8EC6480947F22C3ED94AC
:078B0F00F0EC6480947F226A
:05817800901500EFF07E
:10817D00E5662401FFE43565FAA9077B01A3124DDD
:10818D0036128AE874019013046B7008E9658270E9
:10819D0003EA6583700C7B017A12798490150112C4
:1081AD004D36128AE8128ADF6B7008E9658270031A
:1081BD00EA65836019901500E0856682856583F018
:0E81CD00128AE8AF018A658F66901500E0F017
:0181DB002281
:10850F0053E6F7AA65A9667B01128ADF6401700A38
:10851F00E56665827004E56565837003FF802B78DF
:10852F0067E475F001124D061248D2FF74019013E3
:10853F00046567700AE56965827004E56865837094
:0D854F000975670175681275698443E608B7
:01855C0022FC
:108C8F0053E6F7128ADF6401700AE56665827004A5
:108C9F00E56565837003FF800AAB67AA68A969124F
:068CAF0048D2FF43E60875
:018CB500229C
:03501E00024DF947
:104DF900C0E0C0F0C083C082C0D075D000C000C080
:104E090001C002C003C004C005C006C007901267F4
:104E1900E06003024FE830DF02C2DFE5B05407F576
:104E29006C656A600CE56C656AF56E756B03856C7B
:104E39006AE56B603A156BE56B7034E56E30E00A34
:104E4900E56C20E0057F01128178E56E30E10AE525
:104E59006C20E1057F02128178E56E30E211E56C84
:104E690020E20C90127F7401F0A374F4F0D2153093
:104E7900152690127F74FFF5F0124A0B90127FE00D
:104E89007002A3E07006C215D20C800CE5B030E2C6
:0E4E990007C2157F0412817820D90330D85C3F
:104EA700E5901313543F901533F0C2D8C2D990122E
:104EB70083E0FF901533E0FD6F5403603FEF75F01B
:104EC70004A47E00540CFFED5403FDEF4D241DF5A3
:104ED70082EE3493F583E493901534F06016E0FF87
:104EE7003395E09012818FF0124A0B90127DE4F017
:0C4EF700A37405F0901533E0901283F0D6
:104F030090127DE07002A3E0600A90127D74FFF5B9
:104F1300F0124A0B90127DE07004A3E06401600379
:104F2300024FE8901281E0FCA3E0FD64024C70059F
:104F33007F05024FDE128AEE50047F0180027F005C
:104F4300901281E0FCA3E0FDD39402EC6480948092
:104F530040047E0180027E00EE5F60057F07024F02
:104F6300DE128AF850047F0180027F00128AEE402D
:104F7300047E0180027E00EE5F60047F09805C1284
:104F83008AF840047F0B8053BCFF07BDFE047F06F5
:104F93008049128B0240047F0180027F00C3ED949D
:104FA300FEEC6480947F50047E0180027E00EE5FFD
:104FB30060047F088025128B0C40047F0180027FF0
:104FC30000128B0250047E0180027E00EE5F6004BB
:104FD3007F0A8007128B0C500C7F0C128178901281
:104FE30081E4F0A3F0D007D006D005D004D003D0DD
:104FF30002D001D000D0D0D082D083D0F0D0E03224
:109146007B017A1279848B678A6889698A65896660
:0A915600E490127FF0A3F0C215228E
:067F7D00046105090D116D
:105386003EF583ECF0A3EDF0C3ED9BFDEC9AFCE952
:10539600FF3395E0FEEF25E0FFEE33FE22ED75F0DC
:1053A6002DA424F8F582E43400F583E5822EF582F7
:1053B600E43583F58322E025E0249CF582E4340578
:1053C600F583E0FCA3E0FDEF25E02480F582E434DC
:1053D60005F583E0FEA3E0229005F9124D369015FF
:1053E6001AE09006CDFF75F004024CF1E09005F945
:1053F60075F07DA42445F9740735F0FA7B01024D5A
:10540600363EF583ECF0A3EDF0229006D0EF75F072
:1054160004024CF1E412494C9014D9E025E024250D
:10542600F822E0FF75F005A4F58285F0831248EBBB
:10543600540F22EF75F005A4FF9005F9024D16747E
:10544600FFF5F0124A21FCD3E5F09400EC64809459
:105456008022901423E09006D075F004124CF1E0FF
:1054660022EF9006CD75F004024CF13EF583E0FC88
:10547600A3E0FD2274802FF58274053E222DFFEEF7
:105486003CFEF0A3EFF07C007D0502496EE0FE7560
:10549600F02DA424E1F582E43401F583E5822F2280
:1054A600FF9013F8E0FCA3E0FD22E0246DF582E412
:1054B6003413F583E022900001E92FF9EA35F0FA7A
:1054C600024A62EF25E02425F8760F0876FF22903F
:1054D60013F8EEF0A3EFF022901507E025E0FF9019
:1054E6001506E033FE74B92FF582740422A804A9C8
:1054F60005AA06AB07E0FEA3E0FF22E025E0248034
:10550600F582E43405F583E022FFE4FCFD024CA3BA
:105516007B017A0779459005F9024D36E024DAF5E4
:1055260082E43405F58322E47F2C7E01FDFC124CD7
:1055360097C3024C3E90151EE0FCA3E0FD22F583C6
:10554600E4F0A3F0EF25E022E4F0EF24FAA3F0E084
:10555600FD2461F8E6229005FAE475F005124A0B7F
:1055660090151BE004F02275F02DA424EFF582E4DB
:105576003401F583E5822F22E9D36480F8740B6445
:10558600809822E0FEA3E0FFED25E02425F8A6069C
:1055960008A60722901504EEF0A3EFF0229014243B
:1055A600EEF0A3EFF00D1249D5901424EE229009E7
:1055B60039E0D3648022E4F0ED75F02DA422FFE4F7
:1055C600FCFD7B1FFAF9F8024B2174172FF5827444
:1055D6000622E4FCFD024CA3748F2FF5827406228A
:1055E600EF25E02425F8E6FC08E622AB07AA06A983
:1055F60005A804024C8BE0A3FFE0FCA3E0FD22908B
:105606001413E0FF3395E0FEEF2274962FF58274B3
:10561600003E22F0AF051286DDEF4E22E4F0A374C1
:1056260005F022D39400EE940022124B1478051252
:105636004C65AD07AC06229014DB124D168F8275B1
:1056460083002274002FF58274002274532FF58292
:10565600740622745A2FF58274002225E02425F858
:1056660076080876002225E02425F8E4F608F622D6
:10567600E0FF740BD39F222470F58274053EF583F8
:1056860022124CA3901414024C8B9FEE6480F8EC0B
:045696006480982272
:1086DD00AD07EDB4010F1255B494807E0040037FB9
:1086ED0001227F0022EDB4020F1255B494817E0059
:1086FD0040037F01227F0022EDB4030F1255B49485
:10870D00827E0040037F01227F00221255B49480A7
:0B871D007E0040047F0180027F0022EC
:108E9200E4FFEF25E02400F582E434001255442477
:108EA200B9F582E43404F583E4F0A3F00FEFB42DB6
:018EB200E1DE
:018EB300229C
:108C0F00EF64116022EF6412601DEF641F6018EFB4
:108C1F0064206013EF6428600EEF642B6009EF642B
:0C8C2F00276004EFB42A03D38001C322A5
:1090880090136CE0FF7419D39F500BEF9426500691
:0C909800C3EF940EFF2290136CE0FF2247
:10754100E4FF1254107406F00FEFB405F5E4FF7474
:10755100612FF8E6FE9006D41254147402F0EE90F6
:1075610006D812546B7405F075F004EE9006DC1227
:107571004CF17405F074DA2F125525E4F00FEFB4D5
:1075810004CDE4FF74FC2FF582E43405F583E4F0C7
:1075910074DE2FF582E43405F583E4F00FEFB41BBC
:1075A100E3E4FFEF25E02417F582E43406125544A5
:1075B1002453F582E43406F5837401F0A37490F04A
:1075C100EF25E0248FF582E43406125544245AF560
:1075D10082E43400F5837401F0A3742CF00FEFB44E
:0275E1001EC1C9
:0175E3002285
:109031001255E6D39400EC94004005EF12566C22D1
:0D9041009006CD1254131256221254C9226B
:108E2A00125467125445501112546712554612557E
:108E3A00E94C600EEF125661221255E64C6003129D
:038E4A0054C922E6
:027E4B00AE0780
:107E4D00C21D128C0F50321253A3E060291253A39E
:107E5D001255BC2406F582E434011253AF1255BC01
:107E6D00240EF582E434011253AF1255BC2411F5E2
:107E7D0082E434018037027EC4740BD39E501CEE15
:107E8D00941850171253A3E0600F1253A31255BC50
:107E9D002406F582E434018014801C1253A3E060A3
:107EAD0016ED75F02DA424F8F582E434001253AFCD
:0C7EBD00E4F0AF05029031AF05128E2AF0
:017EC9002296
:055960009014D9EFF0E6
:10596500C212C213C214E075F02DA424F8F9740014
:1059750035F0FA7B019014DB124D369014D9E09086
:1059850006CF1253EBE09014DAF0125410E0B4068F
:105995000D9014DAE0FF9014D9E0FD027E4B9014CF
:1059A500DA1256765014EF9418500FEF6411600414
:1059B500EFB41204D2148002D21330134D12563DA7
:1059C5001248EB60159014DAE0F5827583001254E5
:1059D5001AE6FE08E64E7002D2129014DAE0240EA2
:1059E500FFE433FEA3124D168F828E831248EB70AF
:1059F50003025AD58F828E8312541AE6FE08E64EAC
:105A05006003025AD5D212025AD5201403025AB79E
:105A15009014DAE064117048A3124D16900011122B
:105A250048EB701890001F1248EB70109000271279
:105A350048EB700890002A1248EB6024900011E4AE
:105A450012494C90001FE412494C900027E412497A
:105A55004C90002A12541AE6FE08E64E7002D21245
:105A65009014DAE064127068A3124D1690001212B9
:105A750048EB70189000201248EB70109000281227
:105A850048EB700890002B1248EB6044900012E43C
:105A950012494C900020E412494C900028E4124928
:105AA5004C90002B12541AE6FE08E64E7022D212D4
:105AB500801E9014DB124D169014DAE0FFF5827506
:105AC50083001248EB600912563DE412494CD2128C
:105AD50030120D9014D91253E7125622EF025BD7FC
:105AE5009014D91253E71254454003025BD3125464
:105AF50067E4F0A3F03013289014DAE0FF125502A2
:105B0500FCA3E0D39400EC9400505DEF25E0249CC9
:105B1500F582E434051253D7125629404D025BAF86
:105B2500201403025BBB9014DAE0FF6411703DD3CF
:105B35009005A3E094009005A2E09400502A9005FA
:105B4500D5E094009005D4E09400501C9005CFE07A
:105B550094009005CEE09400500E9005BFE09400AF
:105B65009005BEE09400400280408044EF641270CE
:105B750064D39005A5E094009005A4E09400502A14
:105B85009005D7E094009005D6E09400501C900550
:105B9500D1E094009005D0E09400500E9005C1E04E
:105BA50094009005C0E0940040069014D9E080165A
:105BB5009014D9E080149014DAE01253CE125629CD
:105BC5009014D9E040041256612212566C229014AA
:055BD500D9E01254CAE2
:015BDA0022A8
:10646600C21EEF24FA90151CF0E0FF2461F8E690B6
:10647600151AF01286DDEF4E60747B017A077945B6
:106486001253DE125445505F125467E4F0A3F090A5
:10649600151BF090151BE0FFC39419503B12543F97
:1064A6001248D2540F602C90151C1254B0FEF460A2
:1064B60022EF6E701E90151BA31254931253B4E074
:1064C600600302653C90151BE01253CE125629401C
:1064D60002D21E12555C80BB90151A125421301E32
:1064E6000302659802659E90151AE002657790157D
:1064F6001CE075F07DA42445F9740735F0FA7B019C
:106506001253DE12544540030265A3125467E4F0A9
:10651600A3F090151BF090151BE0FFC3941950696A
:1065260012543F1248D2540F605990151C125493BE
:106536001253B4E06012EE1254951253B4E4F01202
:1065460053E4125622EF802990151BE0FFEE1255F8
:106556006D1253B4E0601EEFD3940A401890151BD9
:10656600A3E012556D1253B4E4F01253E41256220E
:10657600EF1254CA2290151BE01253CE1256294030
:1065860002D21E12555C02651C90151A1254213057
:106596001E06760808760022E4F608F62290151AFA
:0865A600125421760F0876FF64
:0165AE0022CA
:09569A009013F2EFF0A3EDF0F91A
:1056A30012560925E0FBEE33FA745F2BF58274047E
:1056B3003A1253D790140812550F747B2BF582744A
:1056C300043A1253D790140C12550F12557E40030F
:1056D30002595F9013F3E0FF6480949840030259EA
:1056E3005F128C0F500302595F9013F3E0F9FB3301
:1056F30095E0FAEB25E0FFEA33FE74052FF582749B
:1057030004125471745F2FF58274041254077421C8
:105713002FF5827404125471747B2FF58274041272
:10572300540774AB2FF582740312547174052FF56B
:1057330082740412540774C72FF5827403125471D0
:1057430074212FF582740412540774512FF5827457
:105753000312547174AB2FF5827403125407746DE2
:105763002FF582740312547174C72FF582740312D8
:10577300540712547A1253D7FF9013FA1255D8EBE9
:1057830025E0FBEA33FA749C2BF58274053A125335
:10579300D7FFE4FCFD9013FE124CA39013FA124CB6
:1057A3008B74512BF58274033AF583EEF0A3EFF07B
:1057B3009013FE124C8BAD07AC06125395746D2FEC
:1057C300F58274031254079013FE124C8B9013FA54
:1057D3001255F1124B14901402124CA3901402129E
:1057E300552D500302595F90140C124C8B901408E2
:1057F3001255F1124B149013F4124CA39013F4129C
:10580300552D500302595F901408124C8B780C12DB
:105813004C789013F4124C971287FA1254D59013C4
:10582300F3E0FF640B6004EFB4180C9014067404E7
:10583300F0A374CBF0800A9014067403F0A37432BF
:10584300F0901406E0FEA3E01254A6D39FEC9E5002
:1058530009E49013F8F0A3F08015901406E0FEA37A
:10586300E0FFC3ED9FFFEC9E9013F8F0A3EFF090E1
:1058730013F3E0FF640B6004EFB4180F9013F9E027
:1058830025E0F09013F8E033F080169013F8E0FE73
:10589300A3E0FF12548C1254D57D03124980125495
:1058A300D59013F3E01253961256493E1253D71272
:1058B30055C49013F81254F3E4FCFD1256309013C0
:1058C300F3E01253961256491254071256493E12E8
:1058D30053D7FF9013F8EEF0FCA3EFF0FD7B907A23
:1058E300019013F2E0F91253961256513E1253D718
:1058F300C39DEE9C50111254A71253951256511288
:1059030053861255D080271253951255D03E125309
:10591300D71254A6C39FEC9E50171253951255D01D
:10592300125407ED2BFDEC3A1253941256511254B4
:10593300079013F2E0FD1253961255D03E1253D73F
:10594300FF1254D5D394FFEE940F400A9013F874CA
:0C5953000FF0A374FFF09013F8125589B8
:01595F002225
:056C9400901410EFF068
:106C9900AF05EF12539712547AF583E0FFA3E09002
:106CA900141CCFF0A3EFF0AF03EF12539712547AED
:106CB9001253D7FF90141DE02FFF90141CE03EFEE5
:106CC900E4FCFD90141E124CA3E47F1EFEFDFC9013
:106CD900141E1255345003026D9E90141CE0FEA33D
:106CE900E0FFE4FCFD780C124C78A3124C97128754
:106CF900FA9014181255D8901418124C8B780C125B
:106D09004C78901418124CA31256057802C333CE4E
:106D190033CED8F912567D124C8BE47B3F1255CAFB
:106D29007806124C65C004C005C006C00790141847
:106D3900124C8B7806124C65D003D002D001D000DA
:106D4900124B14901414125687C004C005C006C013
:106D5900071256057802C333CE33CED8F912567DC1
:106D6900D007D006D005D004125687E42FFFEE34A1
:106D790008FEE43DFDE43CFC780C124C65D3EF942D
:106D8900FFEE940F40047E0F7FFF901410125421E0
:056D9900A60608A60794
:016D9E0022D2
:108CB6007C007D0B12496EEEA2E713FEEF13FFC395
:108CC60094CBEE648094845005E4FEFF80087435EE
:078CD6002FFF74FB3EFE229C
:0B89C000901506ECF0A3EDF012559AA4
:1089CB00128CB612559A1254DE3E1253D71255C45E
:1089DB009015041254F3EE3395E0FDFC1256301251
:1089EB0054DE1254071254EB3E1253D7FF12559A12
:0189FB002259
:0D72A10090151DEFF0A3ECF0FEA3EDF0FF43
:1072AE00AC02AD031289C090151EEEF0FCA3EFF0F8
:1072BE00FD7B2C7A0190151DE0F91253961256594A
:1072CE003E1253D7C39DEC6480F8EE648098501143
:1072DE0012553B1253951256591253861255DE8093
:1072EE00281253951255DE3E1253D7FF12553BC34B
:1072FE0012569050171253951255DE125407ED2B5D
:10730E00FDEC3A12539412565912540790151DE083
:10731E00FD1253961255DE3E1253D7FF90151EEEF8
:10732E00F0A3EFF0D394FFEE6480948F400A901593
:0E733E001E740FF0A374FFF090151E125589F7
:01734C00221E
:02734D00A9078E
:10734F00E4FBFAE9FD3395E0FCED25E0FFEC33FEBD
:10735F00125610F583E020E4030273EB12557E50B2
:10736F0025E964809498501EED25E0FFEC33FE7400
:10737F009C2FF582740512547112547A1253D72D23
:10738F00FFEE3CFE800A12539512547A1253D7FF28
:10739F00128CB6AA06AB0712539574162FF582748A
:1073AF00053E1253D7D39BEE9A50317C007D05AF2B
:1073BF0003AE0212496EAA06AB07EAC313FAEB1328
:1073CF00FBD394FFEA940F40047A0F7BFFAD0312B7
:1073DF005395125610F583EAF0A3EDF0AF01EF12BB
:0973EF0053971256101253D7FFF8
:0173F8002272
:105BDB00EF24FA90142812555404901423125619DA
:105BEB007003025CAA1255169014281254B090142C
:105BFB0022F0F47003025C8DE0FF64117003025E0F
:105C0B0049EF64127003025E4912543F75F005EFC1
:105C1B0012542D7003025E499006E8E0FF901426A3
:105C2B00F0BF020B901423E0FF901422025CF29061
:105C3B001426E0B40406901422025D00901426E0B2
:105C4B0064036003025E499014221256765013EFE0
:105C5B009418500E1253BC9014241254831255A353
:105C6B00800D901422125501FFA3E0901424CFF065
:105C7B00A3EFF09014231255FC901422E0FB7A0052
:105C8B00801A9006E8E064036003025E49901423D7
:105C9B00E0FF901422E0FB7A00E4FDFC0272A1907D
:105CAB0014281253F2901428125522E0901427F066
:105CBB00129088901422EFF064117003025E49E099
:105CCB00FF64127003025E4912543F75F005EF1228
:105CDB00542D7003025E49901423E0FF12545C9024
:105CEB001426F0B40206A3E0FD02569A125458B4DF
:105CFB000414901427E0FF12734D901423125421B7
:105D0B00A60608A6072212545864036003025E49D4
:105D1B0090142AF0A3F0A3F0A3F0901428E09005C0
:105D2B00131253F6E4901429F0901429E0FFC36486
:105D3B008094994003025DF3900513124D16EF33D7
:105D4B0095E08F82F5837405124CE01248EB540FEB
:055D5B007003025DEA87
:105D6000901429E0FD12539612547AF583E0FFA3B4
:105D7000E090142ECFF0A3EFF0ED12557F5032904B
:105D80001429E0FF648094985027EF125397749C75
:105D90002FF58274053E1253D7FF90142FE02FFF8A
:105DA00090142EE03EFE9014241254881255A380C5
:105DB0000B90142EE0FFA3E0901424CFF0A3EFF09B
:105DC00090142AE0FEA3E09014241255FED312563C
:105DD00090401790142AECF0A3EDF0901429E0FE07
:0A5DE0003395E090142CF0A3CEF0F0
:105DEA00901429E004F0025D34901423E0FF90142B
:105DFA002AE0FCA3E0FDA3E0FAA3E0FB1272A130C3
:105E0A00093DE4901429F0901429E0FFC3648094BA
:105E1A00AD502AEF3395E0FE74722FF58274133E6B
:105E2A00F583E07010901429E012539712547AF512
:0F5E3A0083E4F0A3F0901429E004F080CAC209B9
:015E49002236
:107A9C0090150A12554E2402901509125619602F92
:107AAC0012551690150B1254B0FFF4606790150820
:107ABC00EFF012543F9015081254286057125439A5
:107ACC001254BC127B21C333CE33CED8F9803990FB
:107ADC00150B1253F290150B125522E090150AF06B
:107AEC00129088901508EFF012543F901508E01290
:107AFC00542A602090150AE012543A1254BC127B9E
:107B0C0021C333CE33CED8F9FF901509125421A6D8
:047B1C000608A607AA
:0B7B200022FFAEF0128770EF78022207
:1070690090150E12554E240390150D125619604DA8
:1070790012551690150F1254B0FFF4700302712BBC
:1070890090150CEFF09006F0E06405702512543F5E
:1070990090150C125428700302712B125439900068
:1070A900031254BFAEF07802C333CE33CED8F902FF
:1070B900711390150DE0FF90150C02712690150FB4
:1070C9001253F290150F125522E090150EF01290FE
:1070D9008890150CEFF012543F90150CE012542AC9
:1070E900604090150D12545BB4052C90150EE012FA
:1070F900543AE92FF9EA35F0FA900003124A62AEE0
:10710900F07802C333CE33CED8F9FF90150D12545F
:1071190021A60608A6072290150DE0FFA3E0FD129F
:02712900569A74
:01712B002241
:057724009014DEEFF0FF
:107729009006CF12545F9014E2F01290889014E101
:10773900EFF09014DEE0FF12545CB402089014E2FA
:10774900E0FD02569A9014DE12545BB4041B9014A7
:10775900E2E0FF9014E1E06F705812734D9014DE6F
:10776900125421A60608A607229014E21256765052
:1077790020EF9418501B1253BC9014DF12548390BD
:1077890014DFEEF0A3EFF00D1249809014DFEE80C4
:107799000D9014E2125501FFA3E09014DFCFF0A37E
:1077A900EFF09014DE1255FC9014E2E0FB7A00121F
:0277B90072A1BB
:0177BB0022AB
:108770007C007D69124D97901510124CA390151036
:10878000124C8BE47B64FAF9F8124BAC9015101282
:108790004CA3E47FFF7E0FFDFC901510124C97C395
:1087A000124C54400A901510124CAF00000FFF906D
:0587B0001510124C8BB6
:0187B50022A1
:10883E0074FFF5F0024A0B7403F0A374E8F0A3E59D
:10884E0084F0E4F58422D2C4D2C5D2C2C2C3E4906D
:10885E001545F0FF22EFF0A3ECF0A3EDF0A3024DCF
:10886E0036E5748575F0024A0BE025E044A0F5C2AA
:03887E007F032253
:06945F00C2C253E6FD222B
:066D9F009014301288631D
:106DA50090143912884520C7FDC2C4D2C2D2C5E4A9
:106DB500FF901545F030C3FDAEC1EE124D6B6DDF92
:106DC500006DE2086DE2106DF0186DFA206E022874
:106DD5006E55306E5D3800006DDF026E65EF700632
:106DE500901430128877C2C5026E6B901431E0F5AD
:106DF500C27F0580719015457403F08069EFB40575
:106E05000B901431A3E0F5C27F06805AEF6406703B
:106E15002D901438E0901433700875F001124D1F51
:106E25008003124D161248D2F5C290143612883ED0
:106E3500901436E07002A3E0702C7F078028EFB431
:106E45000706D2C47F09801E9015457405F080168B
:106E55009015457404F0800E9015457406F0800673
:106E65009015457401F0EFB40904C2C3802790154D
:106E750045E0B4030D90143912883E45F0600312C5
:106E85008854901545E06008C2C5D2C4C2C38005C8
:0E6E9500C2C3026DBA20C7FD90143BE0F58425
:016EA30022CC
:0666F100901448128863BA
:1066F70090145012884520C7FDD2C2C2C4D2C5E447
:10670700FF901545F030C3FDAEC1EE124D6B673AF1
:1067170000673D08673D10676218676C206774283B
:10672700678F30679738679F4067AF5067D65800C5
:1067370000673A0267DCC2C5EF70099014481288F7
:10674700770267E2EF640160030267E2901448E0B2
:1067570025E044A1F5C27F040267E2901449E0F501
:10676700C27F0580769015457403F0806EEFB405FF
:106777000B901449A3E0F5C27F06805FEFB40606CD
:10678700D2C57F01805580189015457404F0804B61
:106797009015457406F08043EFB404047F02803BF4
:1067A7009015457405F0803390144BE475F0011291
:1067B7004D1FE5C212493A90144E12883E90144E6E
:1067C700E07002A3E07004C2C280107F02800CD286
:1067D700C47F0980069015457401F0EFB40904C21F
:1067E700C38027901545E0B4030D90145012883EDE
:1067F70045F06003128854901545E06008C2C5D281
:10680700C4C2C38005C2C302670C20C7FD901452DF
:03681700E0F58425
:01681A00225B
:106B7D00901468EFF090146B124D36901469ECF090
:036B8D00A3EDF085
:106B9000757600543FF577543F604BC3744095774A
:106BA000FFE49576FE90146EE0FCA3E0FDC39FEC3D
:106BB0009E50068C748D7580048E748F75126C6B6C
:106BC00060037F022290146912886F901470E07045
:106BD0000690146C12886FC390146FE09575F09056
:106BE000146EE09574F090146EE0F574A3E0F57502
:106BF000D3E5759400E5749400406DE5759440E527
:106C0000749400500F126C6B60037F0222E4F574E1
:106C1000F57580DC901468E0FFA3E0FCA3E0FDA321
:106C2000124D16901436E4F0A37440F0901470E006
:106C3000901438F0126D9F901545E060037F02229A
:106C400074C02575F57574FF3574F574901469E496
:106C500075F040124A0B901470E0709490146C75AB
:0A6C6000F040124A0B026BF07F00B7
:106C6A0022901468E0FFA3E0FCA3E0FDA3124D16F6
:106C7A00901436E574F0A3E575F0901470E0901462
:0A6C8A0038F0126D9F901545E022CE
:1092580090144EE4F0A304F01266F1901545E06016
:07926800037F01227F0022B9
:10916000901544EBF07B017A15794490146EE4F08D
:0A917000A304F0E4A3F0126B7D22CB
:108EB400C007901477E0FFA3E090144ECFF0A3EF27
:108EC400F0D0071266F1901545E060037F01227F20
:028ED40000227A
:10917A00C00790147FE0FFA3E090146ECFF0A3EF36
:0A918A00F0E4A3F0D007126B7D2281
:10855D0000010204081000000304180000000000D0
:10856D001F000000000018040300000000100804A4
:10857D0002010000040A0A11110000010102021C8F
:10858D0000001C0202010100001010080807000085
:0E859D000708081010000020406080A0C0FFFA
:0D936A007F147E00EF1F70011EEF4E70F7A4
:0193770022D3
:10930C007F38128F997F06128F997D0EE4FF02939E
:01931C009EB2
:058F9900901546EFF009
:108F9E00A2AF921FC2AF128F39EF20E7F99015469C
:098FAE00E0FF128FD7A21F92AF61
:018FB7002297
:108F3900A2AF9220C2AF75A0FFC2B5D2B6D2B71206
:0F8F4900936AADA0C2B712936AA22092AFAF0590
:018F580022F6
:059477007F01028F9946
:108FD700A2AF9221C2AF8FA012936AC2B5C2B6D216
:0D8FE700B712936AC2B712936AA22192AF2B
:018FF400225A
:1090DC00A2AF9222C2AF8FA0C2B6D2B7D2B51293B2
:0A90EC006AC2B712936AA22292AF83
:0190F6002257
:0C939E00901547E05FF04DFFF0028F9942
:0291F900AC07C1
:1091FB00A2AF9223C2AF128F39EF20E7F9AF04125F
:06920B0090DCA22392AFEB
:01921100223A
:108D7400901520124D36901520124D161248D260CF
:108D840013901520E475F001124D1F1248D2FF1202
:058D940091F980E222CC
:068A36009014C7124D363A
:108A3C00A2AF9224C2AF129477E4FDFF1293AA90D6
:108A4C0014C7124D16128D74E4FD7F011293AA9077
:108A5C0014CA124D16128D747D107F011293AAA2A6
:038A6C002492AFA2
:018A6F0022E4
:0C93AA00EF75F040A42D2480FF028F9985
:0B93CC00E4F584EF9085A393F5D32215
:047F8300410BAD0001
:1077BC0090145AE0FF75F07090B401124CF1EF2563
:1077CC00E02583AF8222E475F001124A0B90145C21
:1077DC00E475F001024A0BFE7A0679CD7B01901418
:1077EC009E7402F0A37470F022AFF0FEE0FCA3E0F4
:1077FC00F5828C83E493FD22901456F0A3EFF0E411
:10780C0090145CF0A3F0227E007C027D7012496E15
:10781C0074012FF974B43EFA7BFF22EBF0AC07A293
:10782C00AFE433A3F0C2AF2275F070EE90B4011246
:10783C004CF1EE22E475F001024A21EDFFAD04EDAE
:07784C00CFF0A3EFF0E422EE
:06946500E4900BADF022C3
:07941900900BAD7401F0227D
:1085F8009015357402F0E4A3F01294117EB47F0054
:108608007A1579351286377EFF7F917A1579361279
:108618008637128D047E027F707D007B017A067991
:0F862800CD124DC41275411292127F1E028B8328
:0E8637007B0190149EE4F0A304F0128A7022DE
:108FB800E5B030E01190FF91E493F4600990B400BB
:0F8FC800E493640260031285F8E49006CBF02274
:058B8300901537EFF032
:108B8800129411E4901538F0901537E0FFA3E0FE39
:108B9800C39F50141278341277CB1277E3128A707D
:0B8BA800901538E004F080E0028D041E
:1092C400300B0B900BADE07002D20ED21722D20AF3
:0492D400126EA42250
:035003000292C452
:0A8D99009006CBE0FFC3941E5018B3
:108DA3009006CFE0901548F012781378CD7C067DBD
:088DB300017E027F701248AC42
:038DBB00C21722BA
:1090A4009006CBE0C3941E50121294119006CB127A
:0C90B40077BF1277E3128A70128D04223D
:10921200A2AFE433901549F0C2AF1290A4C21790E6
:079222001549E024FF92AFA3
:019229002222
:0878530090143DEDF0A3EBF0F1
:10785B00A3E004F0901442EFF0A3EBF090143DE0A2
:10786B00FF901442E0FED39F505B1278341277CB1B
:10787B00901444F0A3EFF09014431277BF9014468A
:10788B00F0A3EFF0E4901440F0A3F09014461278BC
:10789B00409014441277F5127FBD9014441277DC9C
:1078AB009014401277DCC3901441E0947090144014
:1078BB00E0940240D6128D04901442E004F0A3E051
:1078CB0004F00278679006CBE0FF90143EE0D39F64
:0B78DB005009A3E0C39F4003128D99E9
:0178E600227F
:0F6A6300901454EDF0901453EFF0901455EBF0A5
:106A720090145AEFF0A3EBF0901454E0FF90145AE4
:106A8200E0D39F4003026B38A31277BF12780490C1
:106A9200145CE0FEA3E0FFC39470EE9402501A90DF
:106AA20014561277F8743D2FF58274093EF583ED82
:106AB200F09014561277D280D61277BC901458F008
:106AC200A3EFF090145B1277BF1278049014561261
:106AD20078409014581277F5127FBD9014581277AF
:106AE200D2C390145DE0947090145CE0940240DC98
:106AF2001277BC90145812780790145CE0FCA3E063
:106B0200FDC39470EC9402501D901458127840AF5B
:106B1200F0FE743D2DF58274093CF583E0FD127F91
:106B2200BD1277D980D3128D0490145AE004F0A3D9
:106B3200E004F0026A7A9006CBE0FF901455E0FE82
:106B4200D39F5020901453E0FDA3E0C39DFDE49435
:106B520000FCEE7A002DFDEA3CFCC3ED9F7480F848
:106B62006C9850139006CBE0FF901453E0D39F50E3
:0A6B720009A3E0C39F4003128D99B0
:016B7C0022F6
:037DCB0090148190
:107DCE0012782712945F901487127847901483F0DC
:107DDE00901481E0FF901487E0FCA3E0FD7B017A14
:107DEE0009793D9014771277ED128EB49014877442
:107DFE000275F070124A0B901483E0FF127813A3F1
:107E0E00124D36129411901484124D16AE02AF011B
:107E1E007A09793D1277E8128A70128D04901483D4
:107E2E00E004F0E0C3941E40A7128D9990139FE0DA
:0C7E3E00FF129378901482E024FF92AFB2
:017E4A002215
:0380A3009014A78F
:1080A60012782712945F9014AA1278479014A9F0B8
:1080B6009014A9E0FFC3941E503E75F070EF12773E
:1080C600C4FE9014ACF0FAA3EFF0FB9014A7E0FF07
:1080D6009014AAE0FCA3E0FDA9037BFF90147F1295
:1080E60077ED12917A9014AA740275F070124A0B09
:1080F6009014A9E004F080B890139FE0FF129378E3
:088106009014A8E024FF92AFE1
:01810E00224E
:10932D00E0FEA3E0F5828E8322E475F001024A0B84
:108BB3007E0F7FDB900FB4EEF0A3EFF0900FB0EEDB
:108BC300F0A3EFF07E107FA3900FB6EEF0A3EFF0CB
:108BD300900FB2EEF0A3EFF0E490116BF0C22522F8
:03500F00027A0C16
:107A0C00C0E0C0F0C083C082C0D075D000C000C040
:107A1C0004C006309825C298900FB012932DE599AA
:107A2C00F0900FB0129336FCE5F0B4A30EECB4104A
:107A3C000A900FB0740FF0A374DBF03099419011E1
:047A4C006BE0603754
:107A5000900FB612932DE090154AF0C299F59990C7
:107A60000FB8E599F090116BE014F0900FB61293F7
:107A700036FCE5F0B46B14ECB41110900FB6741032
:057A8000F0A374A3F067
:107A85008004C299C225D006D004D000D0D0D082BF
:077A9500D083D0F0D0E032F5
:10919400900FB4E0FEA3E0FF900FB0E06E7003A365
:0A91A400E06F60037F01227F0022CC
:108DBE00900FB412932DE0FF900FB4129336900FD4
:108DCE00B4E0B4100FA3E0B4A30A900FB4740FF084
:048DDE00A374DBF0AF
:018DE200226E
:1060AA004C00500049002000540043560050756CC3
:1060BA007320313A2573257320323A2573257300EC
:1060CA00333A2573257320343A2573257320353ADC
:1060DA00257325730043562031303A2573257320E2
:1060EA0031313A257325730031323A2573257320ED
:1060FA0031333A2573257331343A257325730043B6
:10610A006F6E747261737420256420006F66660076
:10611A00363700363738003637383900506F6C79E1
:10612A0070686F6E792025732000546F67676C65FD
:10613A00005375737461696E004C3A2573202563A8
:10614A00657600523A257300526164696F3A256494
:10615A002025733A257320257320004B59006B794B
:10616A00004356313A252D3364204356323A25648A
:10617A0020004356313A252D3364204356323A25BE
:10618A007320006C6F6300616263646566676869A7
:10619A006A6B6C6D6E6F70717273747576777879DD
:1061AA004142434445464748494A4B4C4D4E4F505D
:1061BA00515253545556575859FF60AA02FF60ACC2
:1061CA0003FF60AE04FF60B000FF60B206FF60B478
:1061DA0005FF60AA02000600070008000900050082
:1061EA0009000D00110007FF947C0008FF9471005C
:1061FA000CFF9481000DFF94430102FF9486010372
:10620A00FF944A0107FF948B0108FF9451010CFF88
:10621A009490010DFF94580006FF681B0008FF9038
:10622A00C0000BFF8B16000DFF7B2B0105FF86912B
:10623A00010DFF7D4A0006FF94950007FF94200098
:10624A000CFF949A000DFF94270103FF949F010409
:10625A00FF942E0109FF94A4010AFF9435010EFF51
:10626A0094A9010FFF943C0009FF92850109FF924E
:10627A0085000AFF8ED6010AFF8ED60002FF93D749
:0A628A00000AFF8E4D0102FF93850C
:107F87004311AD00000041126102C1274112660191
:107F970041123800411267000C0FFF6116FF611A8A
:107FA700FF611DFF61210609FF6134FF613B010885
:057FB70001021B0001A6
:105E4A00EDFF3395E0FE75F003EF124CF1EE75F0BD
:105E5A0003A42583F583222491F9E43461FA124DCF
:105E6A00360248D27A12794E9014CA7B01124D3604
:105E7A007A12793B2290117C75F003ED124CF1EC09
:105E8A0022EFF0A2AFE433A3F0128C3BC2AF901220
:105E9A00677401F0EF75F005A4FF9011AD024D167D
:105EAA007BFF9013AA024D369011AD124D36901217
:105EBA0038E075F002A4FFAEF024DFF974613EFA0F
:105ECA007BFF9011B5024D36124D16124D4B9013B1
:105EDA00AD124D367B0122E02491F9E43461FA22B5
:105EEA00FD901268124D16124A37AEF078022290CF
:105EFA0011B0124D160248D2124D16124D4B901384
:105F0A00B3024D3690148A124D16740212493A7B26
:105F1A00FF7A6179C3227BFF90119C024D367B0187
:105F2A009011B0024D367B017402AD079014E7F070
:105F3A0022901493124D1690000322124D1690616E
:105F4A00A9D3E99582EA958322740312493A7BFF21
:105F5A007A6179C722F9E43461FA7BFF90127A02F6
:105F6A004D369013ADF0A3EFF022EDFF3395E0FE2E
:105F7A002275F005EFA429F9EA35F0FA0248D29021
:105F8A0011CC024D36EFF09011B5124D16024A3778
:105F9A0024FCF974063EFA7B01024D36D3EF648085
:105FAA009480229014B1E0FFA3E09013ADCFF0A348
:105FBA00EFF022124D16124D4B9013B9124D367B4B
:105FCA00012275F003A4246EF582E43412F58322CB
:105FDA0075F005A424D1F582E43411F5832275F015
:105FEA0005A424CFF582E43411F5832275F005A4C3
:105FFA0024D0F582E43411F58322E075F07DA424DF
:10600A0045F9740735F0FA22E0FEA3E090117C7599
:10601A00F00322901266F07BFF227BFF7A6179CB34
:10602A0022124A62FFAEF0D39400EE94FE2290133D
:10603A00B0024D3674E72FF974613EFA9012682265
:10604A00124D16C3E9949122900939E0C364802263
:10605A00E075F003A42409F8024CFDE024FF92AF96
:10606A00E4901267F0229013BC124D367A12794EE0
:10607A002224D0F58274063EF58322124D1674FF4F
:10608A009061A26B22124D1674FF9061A36B2224B9
:10609A00D4F58274063EF583227B017A12793B227B
:107BBA00E490119BF090119AF09011A1F09011A00D
:107BCA00F090119FF09011A2F07B017A077945900D
:107BDA0011AD124D367BFF7A6179DF125ECC7A6184
:107BEA0079E7901268124D367A61799190127A1279
:107BFA005E689011B8F0E4A3F0901233F0FF125FC0
:107C0A0019EF125FCC124D360FEFB404F1E4901263
:107C1A003AF090124DF0901260F0901263F09012C8
:107C2A0065F09011A4F09011A6F09011A8F09011AF
:067C3A00AAF09011ACF06D
:017C40002221
:06946B00E49011B4F022B0
:10823F00901539EEF0A3EFF0AF051DEF60539015D9
:10824F0039E0FEA3E0F5828E83A3A3124D3F901178
:10825F00B4E0FF125FDA124D36901539E0FAA3E061
:10826F00FBF5828A83E493FEEF125FE8EEF08B82D8
:10827F008A83740193FF9011B4E0125FF6EFF090D0
:10828F0011B4E004F0901539E475F005124A0B8033
:02829F00A72214
:108EF800125EF9FE125FE8E0FFEE125FF6E0FD1287
:108F080093AA125EF9125FDA124D169011C9024D3A
:018F18003622
:1090F7009011B0124D167401124918125EF9FF90C3
:0B91070011B4E0B50704E412493A225D
:108C6600D3ED6480948040047401800274FF12493D
:108C7600181248D2FFB4FF03E4800A9014E7E0FE1E
:098C8600B50705EE1412493A226B
:109285007B017A1279617408125F34128C66901230
:0692950061E0FF0293CC32
:108ED6007B017A097939AD079014E77404F0128C96
:108EE60066E4901238F0126004125EB212603E021E
:028EF6004D36F7
:0B93D7007A09793A125F30128C66228E
:108E4D007A09793C125F30128C66E4901367F090CA
:108E5D0013A4F07F0512922A7F011291127F031243
:038E6D009112223D
:0D9385007B017A09793B125F32128C66225F
:0994000090119C124D16024D91D1
:108FF5009012667401F07A7E79CA125F207A9079B0
:0E90050013125F897A9079F790126B024D3644
:109013009012667402F07A627994125F207A9079E2
:0E9023004E125F897A9079F790126B024D36EB
:10904E00740312601D7A79797B125F227A90796BA4
:0D905E00125F897A9079F790126B024D36FF
:10906B00740412601D7A877928125F227A8F7959DE
:0D907B00125F897A9079F790126B024D36E2
:108F59009012667405F07BFF7A897944125F227A50
:108F69008F7979125F897A9079F790126B024D3671
:108F79009012667406F07BFF7A8179DC125F227A9F
:108F89008F79F5125F897A9079F790126B024D36D5
:0288C300AD07FF
:1088C500ED3395E0FEEF7802C333CE33CED8F99081
:1088D50014CD125F9AAF05EF3395E0FE90114F125C
:1088E5005E50124D169014D0124D369014CD125E76
:1088F500FCB40209125F539014D0124D3602500396
:10898300125FA67BFF40067A6179D380047A61790E
:10899300CF9011BA125E4A124D36125F749011BA1B
:1089A300125E50125F3E1248EBFCEF7802C333CEE7
:0D89B30033CED8F912607BECF01250032295
:05947C00E4FD028983FC
:059481007D010289835A
:059486007D0202898354
:05948B007D030289834E
:059490007D0402898348
:107CC70090148A124D36125FA6402890148A125ECD
:107CD700FC24FE600A1460091460082404706180A3
:107CE70026800090148A124D16740412493A1260C5
:107CF70024804790148A125EFC24FE600F146011E2
:107D070014602E24047039125F53802E125F0E8088
:107D170029901490E075F003A4246DF582E43411E2
:107D2700F583125EFCD3648094EB4014125F0E80DF
:107D37000990148A124D16125F5390148D124D3606
:037D4700025003E4
:0287B600AC070E
:1087B800125F74EF7802C333CE33CED8F99014D356
:1087C800125F9A125F7490114F125E50124D1690FC
:1087D80014D6124D36AF049014D6124D1690148D3F
:1087E800124D36901490EDF09014D3124D16127C61
:0187F800C7B9
:0187F900225D
:059495007D0A0287B60C
:05949A007D0B0287B606
:05949F007D0C0287B600
:0594A4007D0D0287B6FA
:0594A9007D0E0287B6F4
:106FA200125FA64043125E7F125E58A3E475F001A1
:106FB200124A0B30267C125E7F125E581260857078
:106FC20008E965827003EA65836015125E7F125ECE
:106FD2005812608F7008E965827003EA6583705207
:106FE2007BFF7A6179A48041125E7F125E58A3749E
:106FF200FFF5F0124A0B302639125E7F125E5812EC
:1070020060857008E965827003EA65836015125E27
:107012007F125E5812608F7008E965827003EA651C
:1070220083700F7BFF7A6179A1125E7F125E581224
:107032004D36125E7F125E58125F4540087BFF7A22
:107042006179A98018125E7F125E58124D16C390A4
:107052006191125F4C500F7BFF7A617991125E7FD2
:07706200125E58124D3622A8
:10835D0090153BECF0A3EDF0D226126FA290153BD9
:10836D00126012125E5412604AFD90153BE0FAA3A2
:10837D00E0FB7802C333CE33CED8F9240FF58274E7
:10838D00073EF583EDF0126016EB124CF1EA125E2A
:10839D0058125EFCC3648094EC500B90153BA3E027
:0983AD002405FF1288C3025003ED
:079420007D057C0002835D65
:079427007D067C0002835D5D
:07942E007D077C0002835D55
:079435007D087C0002835D4D
:07943C007D097C0002835D45
:108B4D0090153DECF0A3EDF0C226126FA290153DED
:108B5D00126012125E5412604AFD90153DA3E0782A
:108B6D0002C333CE33CED8F924CFF58274063EF549
:068B7D0083EDF00250033D
:06947100E4FDFC028B4D3E
:079443007D017C00028B4D4E
:07944A007D027C00028B4D46
:079451007D037C00028B4D3E
:079458007D047C00028B4D36
:10681B00125FA650030268A1125EA4740190074593
:10682B006B7008E965827003EA6583701F90093904
:10683B00E014601014601014600F240360030269ED
:10684B002E0268FA0269218069026902125EA47441
:10685B00019007C26B7008E965827003EA6583706B
:10686B0003026921125EA4740190083F6B7008E962
:10687B0065827003EA658370028037125EA474012F
:10688B009008BC6B7008E965827003EA658360034E
:10689B0002692E02692A125EA474019007456B707F
:1068AB0008E965827003EA65837011126052948364
:1068BB0050089012387403F08069803B125EA47408
:1068CB00019007C26B7008E965827003EA658370FB
:1068DB0002804C125EA4740190083F6B7008E9654E
:1068EB00827003EA65837012126052948150089093
:1068FB0012387401F0802CE48025125EA474019090
:10690B0008BC6B7008E965827003EA65837014122A
:10691B006052948250089012387402F08005E49013
:10692B001238F09012381260047B01125EB21260C2
:05693B003E124D362262
:1090C000125FA640079012377401F022E490123725
:0C90D000F07F031283027F3912922A22E3
:108C3B0090127A124D16C3906191125F4C401090B6
:108C4B00127A125F45500890127A12604AFF2290F6
:0B8C5B00127A124D16C3E994AAFF2202
:028B1600AE07A8
:108B1800128C3BD3EE64809480401274AA2F125FAB
:108B28005F125EA4125F7B54F04401801274912F8F
:108B3800F9E43461125F63125EA4125F7B54F01291
:058B4800493A02500350
:037B2B0090154B67
:107B2E00125F8F24FAFFE5F034FFFE90154BE0D381
:107B3E006480948090126E75F003EF400A125E54CA
:107B4E00A3E475F0048009125E54A374FF75F0FC73
:107B5E00124A0B90126E125E50124D169061CB129D
:107B6E005F4B400C12602490126E125E50124D3616
:107B7E0090126E125E50124D16C39061C3125F4C7E
:107B8E00500C125F1990126E125E50124D369012FA
:107B9E006E125E50125F3E1248EB125EEAC333CE97
:0C7BAE0033CED8F9126099EDF0025003BC
:10864500EF124D6B866501866F028679038683047A
:108655008688FC867EFD8674FE866AFF0000868D10
:108665007E007F01227EFF7FFF227E007F10227E1B
:10867500FF7FF0227E007F40227EFF7FC0227E00AA
:0C8685007FFF227EFF7F0122E4FEFF2227
:0386910090153F02
:10869400125E8BE92FF9EA35F0FA90153FE0FF12EC
:1086A4008645900001EE8FF0124A9A900001126004
:1086B4002B4008900001E4F5F08011C3EF94CFEE55
:1086C4009403400B900001740375F0CF124AE71233
:0886D40050039015401260658F
:0186DC00227B
:037D4A0090149101
:107D4D00125E8BE92FF9EA35F0FA901493124D3645
:107D5D00125EEBC333CE33CED8F924D9F974063E77
:107D6D00FA7B01901496124D36901491E0FF128615
:107D7D0045125F3BEE8FF0124A9A90000312602B72
:107D8D004013125F3BE4F5F0124AE7901496125F30
:107D9D003E7402801CC3EF94CFEE9403400B125F30
:107DAD003B740375F0CF124AE7901496125F3E7440
:0D7DBD000512494C1250039014921260659B
:017DCA002296
:1078E700900723125EE17BFF90118B125E68901167
:1078F700A3F0900727E090118E125E619011A5F01A
:1079070090072BE0901191125E619011A7F09007FC
:107917002F125EE1901194125E689011A9F0900702
:1079270033125EE1901197125E689011ABF0E4FD9F
:10793700125F74EF7802C333CE33CED8F92424F51F
:107947008274073EF583E0601024FD600C14600E1E
:1079570024027019125F198008125F5880031260A1
:1079670024125F7490116D125E50124D360DED6446
:037977000570BDDB
:01797A0022EA
:107ECA00127C417A6079B7125EAA9011BA125ED218
:107EDA007A1279391260389011BD125F027A1279DA
:107EEA004C9013B6125E751250867A6079CA125E89
:107EFA00AA9011C0125ED27A12795F12603890117C
:107F0A00C3125F027B017A1279629013B6124D3660
:107F1A009011C6125FBD7A1279641260701250868F
:107F2A00125E6E128A3612946B7E617FEF7D0A12A0
:0C7F3A00823F7A11799A125F28028EF8BB
:10797B00E4901237F07F031283027F3912922A129E
:10798B0078E77BFF7A6079DF125EAC90116D125E47
:10799B00D27A1179A3126038901170125F027B01B9
:1079AB007A1179A59013B6125E771250867BFF7A07
:1079BB006079F2125EAC901173125ED27A1179A7D4
:1079CB00126038901176125F027B017A1179A990BF
:1079DB0013B6124D36901179125FBD7A1179AB1235
:1079EB006070125086125E6E128A3612946B7E6233
:1079FB007F3F7D0A12823F7A11799F125F28028E98
:017A0B00F882
:108728007BFF7A617909125EAC901261E0FFE41276
:108738005F6C1260A31250867BFF7A6079B0125E7C
:10874800AC7B017A12794E125086125E6E128A360E
:1087580012946B7E627F717D0112823F7B017A11D8
:0887680079A0125F2A028EF8CD
:108944007BFF7A617926125EAC900939E075F003F9
:10895400A4240FF8124CFD125ED87A12793B1250FF
:1089640086125E6E128A3612946B7E627F7B7D0164
:0F89740012823F7B017A1179A1125F2A028EF8DD
:1081DC007BFF7A617943125EAC90093A12605A9037
:1081EC0013AD124D3690093CE060047F5280027F43
:1081FC00729013B0EFF01260A31250867BFF7A617D
:10820C00794D125EAC90093B12605A125ED87A120C
:10821C00794E125086125E6E128A3612946B7E6202
:10822C007F857D0312823F7B017A1179A2125F2A2E
:03823C00028EF8B7
:107C41009006CF125EE17BFF90117C125E6890126C
:107C510039F09006D3125EE190117F125E689012A6
:107C61004CF09006D7125EE1901182125E6890127C
:107C71005FF09006DB125EE1901185125E68901252
:107C810062F09006DF125EE1901188125E68901238
:107C910064F0E4FD125F74EF7802C333CE33CED8C3
:107CA100F912607BE07BFFB406067A6179D3800428
:107CB1007A6179CF125F749011BA125E50124D360B
:057CC1000DEDB405CF3C
:017CC600229B
:108DE30090119C124D16EB8A8389827BFF7A6279FC
:108DF30094F4700A749465827004746265837003DA
:048E030012940022A3
:1082A100E4901541F0901541E0FFC364809499502A
:1082B1004F901238E075F07D900745124CF1EF3385
:1082C10095E0FE75F005EF124CF1EE75F005A42571
:1082D10083F583E0540F9015416009E025E0240700
:1082E100A3F08007E025E02406A3F07F03128302B8
:1082F100901542E0FF12922A901541E004F080A50A
:018301002259
:10629400901237E0600D7F031283027F3812922A36
:1062A4001282A190136CE0FFC39419400BEFD394B6
:1062B400265005EF24F2800490136CE09014AFF0A4
:1062C4009014AFE0FF128C0F500890116CE0901402
:1062D400AFF09014AFE0FF642C6004EFB429089091
:1062E400116CE09014AFF09014AFE0FF90116CF0DB
:1062F400125EA475F005EFA4F58285F0831248EBD5
:10630400540F9014AF600CE024AA125F5FC3E994A9
:10631400AA800A125EE1125F64C3E994919014AEFC
:10632400F09014AEE0125E9FE92F125F81C4540F07
:106334009014B0F0900001124A62FF9014B1E5F09D
:10634400F0A3EFF0900003124A62FF9014B3E5F05B
:10635400F0A3125F8F24FA125EEAC333CE33CED891
:10636400F9126099E024FE600A14600C14600E2493
:10637400047016125F198008125F5880031260249B
:1063840090126E125E4A124D3690127A125EFC9092
:1063940011B8F07BFF7A617952125EAC125F91FF03
:1063A400E5F0125F6C901237E07BFF60067A61794A
:1063B4006580047A6179689013AF124D367B017A57
:1063C4001179B89013B2124D36ED125FCC124D16FE
:1063D400124D4B9013B5124D361260A31250861213
:1063E4005EEBC333CE33CED8F924DCF58274063E9B
:1063F400F583E07BFFB4051B7A61796B125EAC1206
:106404005FAD9014B3E0FFA3E09013AFCFF0A3EF20
:10641400F080127A61797C125EAC125FAD7A617998
:106424008DA3124D367B017A12794E125086C39099
:1064340013A1E094109013A0E09427400D125E6E17
:10644400128A36E49013A0F0A3F012946B7E627F5C
:10645400217D0612823F7B017A11799B125F2A0209
:026464008EF8B0
:03000000024000BB
:03000300025003A5
:03000B000250069A
:030013000250098F
:03001B0002500C84
:0300230002500F79
:03002B000250126E
:0300330002501563
:03003B0002501858
:0300430002501B4D
:03004B0002501E42
:0300530002502137
:03005B000250242C
:0300630002502721
:03006B0002502A16
:0300730002502D0B
:03007B0002503000
:03008300025033F5
:03008B00025036EA
:03009300025039DF
:03009B0002503CD4
:0300A30002503FC9
:10400000787FE4F6D8FD9000007F007E20E4F0A3E6
:0A401000DFFCDEFA758179024055ED
:10401A0002409AE493A3F8E493A34003F68001F2E2
:10402A0008DFF48029E493A3F85407240CC8C333A7
:10403A00C4540F4420C8834004F456800146F6DF76
:10404A00E4800B0102040810204080907F46E47E41
:10405A00019360BCA3FF543F30E509541FFEE4936B
:10406A00A360010ECF54C025E060A840B8E493A332
:10407A00FAE493A3F8E493A3C8C582C8CAC583CA5D
:10408A00F0A3C8C582C8CAC583CADFE9DEE780BE15
:017FBC0000C4
:1047DC00E709F608DFFA8046E709F208DFFA803EBF
:1047EC0088828C83E709F0A3DFFA8032E309F608AC
:1047FC00DFFA8078E309F208DFFA807088828C8314
:10480C00E309F0A3DFFA806489828A83E0A3F608C7
:10481C00DFFA805889828A83E0A3F208DFFA804CA1
:10482C0080D280FA80C680D4806980F28033801078
:10483C0080A680EA809A80A880DA80E280CA8033E1
:10484C0089828A83ECFAE493A3C8C582C8CCC58359
:10485C00CCF0A3C8C582C8CCC583CCDFE9DEE78029
:10486C000D89828A83E493A3F608DFF9ECFAA9F0A8
:10487C00EDFB2289828A83ECFAE0A3C8C582C8CCFE
:10488C00C583CCF0A3C8C582C8CCC583CCDFEADE17
:10489C00E880DB89828A83E493A3F208DFF980CC79
:1048AC0088F0EF60010E4E60C388F0ED2402B40472
:1048BC000050B9F582EB2402B4040050AF23234519
:0648CC00822390482C73CA
:1048D200BB010689828A83E0225002E722BBFE02E4
:0948E200E32289828A83E4932217
:1048EB00BB010CE58229F582E5833AF583E0225082
:1048FB0006E92582F8E622BBFE06E92582F8E222CC
:0D490B00E58229F582E5833AF583E49322E5
:10491800BB010989828A83F8E028F022500327F72F
:1049280022BBFE05F8E328F3228A838982F8E49300
:02493800282233
:10493A00BB010689828A83F0225002F722BBFE015C
:02494A00F32256
:10494C00F8BB010DE58229F582E5833AF583E8F0A1
:10495C00225006E92582C8F622BBFE05E92582C84D
:02496C00F22235
:10496E00EF8DF0A4A8F0CF8CF0A428CE8DF0A42E5D
:02497E00FE2217
:10498000BC000BBE0029EF8DF084FFADF022E4CC1B
:10499000F875F008EF2FFFEE33FEEC33FCEE9DECE4
:1049A000984005FCEE9DFE0FD5F0E9E4CEFD22ED2A
:1049B000F8F5F0EE8420D21CFEADF075F008EF2F74
:1049C000FFED33FD4007985006D5F0F222C398FD65
:0549D0000FD5F0EA2202
:1049D500C2D5EC30E709B2D5E4C39DFDE49CFCEEFD
:1049E50030E715B2D5E4C39FFFE49EFE124980C3AC
:1049F500E49DFDE49CFC800312498030D507C3E4A7
:064A05009FFFE49EFE226B
:104A0B00C5F0F8A3E028F0C5F0F8E5821582700236
:064A1B001583E038F022D3
:104A2100A3F8E0C5F025F0F0E58215827002158348
:064A3100E0C838F0E822A5
:104A3700BB010A89828A83E0F5F0A3E0225006874A
:104A4700F009E71922BBFE07E3F5F009E31922890C
:0B4A5700828A83E493F5F0740193223F
:104A6200BB0110E58229F582E5833AF583E0F5F092
:104A7200A3E0225009E92582F886F008E622BBFE6F
:104A82000AE92582F8E2F5F008E222E5832AF583B5
:084A9200E993F5F0A3E993227A
:104A9A00BB010DC58229C582C5833AC583024A0B6B
:104AAA005011C58229F808E5F026F618F5F0E582D6
:104ABA0036F622BBFE11C58229F808E225F0F5F088
:104ACA00F218E23582F222F8E58229F582E5832A94
:0D4ADA00F58374019325F0F5F0E493382284
:104AE700F8BB0111E58229F582E5833AF583E8F001
:104AF700E5F0A3F0225009E92582C8F608A6F022BE
:0D4B0700BBFE09E92582C8F2E5F008F222A4
:0D4B1400EF2BFFEE3AFEED39FDEC38FC22F0
:104B2100E88FF0A4CC8BF0A42CFCE98EF0A42CFC33
:104B31008AF0EDA42CFCEA8EF0A4CDA8F08BF0A4B1
:104B41002DCC3825F0FDE98FF0A42CCD35F0FCEB10
:104B51008EF0A4FEA9F0EB8FF0A4CFC5F02ECD39D5
:0F4B6100FEE43CFCEAA42DCE35F0FDE43CFC2242
:104B700075F008758200EF2FFFEE33FECD33CDCCFC
:104B800033CCC58233C5829BED9AEC99E58298407F
:104B90000CF582EE9BFEED9AFDEC99FC0FD5F0D65C
:104BA000E4CEFBE4CDFAE4CCF9A88222B800C1B986
:104BB0000059BA002DEC8BF084CFCECDFCE5F0CBC4
:104BC000F97818EF2FFFEE33FEED33FDEC33FCEBFD
:104BD00033FB10D703994004EB99FB0FD8E5E4F9B8
:104BE000FA227818EF2FFFEE33FEED33FDEC33FCA5
:104BF000C933C910D7059BE99A4007EC9BFCE99A99
:104C0000F90FD8E0E4C9FAE4CCFB2275F010EF2FDD
:104C1000FFEE33FEED33FDCC33CCC833C810D707DD
:104C20009BEC9AE899400AED9BFDEC9AFCE899F818
:0E4C30000FD5F0DAE4CDFBE4CCFAE4C8F922AB
:1087FA00C2D5E830E70FB2D5E4C39BFBE49AFAE4AA
:10880A0099F9E498F8EC30E717B2D5128830124B90
:10881A00ACE4C39BFBE49AFAE499F9E498F8800380
:10882A00124BAC30D50DE4C39FFFE49EFEE49DFDE0
:04883A00E49CFC229C
:104C3E00EB9FF5F0EA9E42F0E99D42F0EC6480C8ED
:064C4E0064809845F0228D
:104C5400EB9FF5F0EA9E42F0E99D42F0E89C45F0B6
:014C6400222D
:104C6500E8600FECC313FCED13FDEE13FEEF13FF2D
:034C7500D8F12251
:104C7800E8600FEFC333FFEE33FEED33FDEC33FC9A
:034C8800D8F1223E
:0C4C8B00E0FCA3E0FDA3E0FEA3E0FF229C
:0C4C9700E0F8A3E0F9A3E0FAA3E0FB22A0
:0C4CA300ECF0A3EDF0A3EEF0A3EFF02284
:104CAF00A8828583F0D083D082124CC6124CC612D4
:104CBF004CC6124CC6E473E493A3C583C5F0C583F9
:104CCF00C8C582C8F0A3C583C5F0C583C8C582C84F
:014CDF0022B2
:104CE000F5F0C582A4C582C5F0C583A42583F583EC
:014CF00022A1
:0C4CF100A42582F582E5F03583F58322CE
:094CFD00E6FB08E6FA08E6F922DC
:104D0600FAE6FB0808E6F925F0F618E6CA3AF622AE
:094D1600E0FBA3E0FAA3E0F9229E
:104D1F00F8E0FBA3A3E0F925F0F0E582158270021D
:074D2F001583E0FA38F022C1
:094D3600EBF0A3EAF0A3E9F0227E
:0C4D3F00E493FB740193FA740293F922D0
:104D4B00BB010789828A83024D165005E9F8024C94
:104D5B00FDBBFE05E9F8024DF089828A83024D3FC7
:104D6B00D083D082F8E4937012740193700DA3A3D7
:104D7B0093F8740193F5828883E4737402936860EB
:064D8B00EFA3A3A380DFEB
:064D91008A838982E473AD
:104D9700EC8EF0A4CCC5F0CCCDF8EFA4CEC5F02DA9
:104DA700FDE43CFCE8A42EC8C5F03DFDE43CFCEF67
:0D4DB700A4FFE5F028FEE43DFDE43CFC22F5
:10502100E56F24AAF582E43413F583E0056F22903D
:1050310013A73007039013AAE475F001124D1F0264
:1050410048D22000E97F2ED2008018EF540F24901F
:10505100D43440D4FF30040BEF24BFB41A00500302
:105061002461FFE570600215700573E57370020538
:105071007230070E9013A7E475F001124D1FEF0275
:10508100493A028CDD7403D2078003E4C207F56F4D
:105091009013A7124D36E4F570F572F573E5706063
:1050A100077F2012506480F57571FFC201C200C2F2
:1050B10002C203C205C206C208125030FF700D3091
:1050C10007057F00125075AF73AE7222B4255FC21F
:1050D100D5C204125030FF24D0B40A00501A75F022
:1050E1000A787030D50508B6FF0106C6A426F62059
:1050F100D5047002D20380D924CFB41A00EF500432
:10510100C2E5D204025276D20180C6D20080C0D25A
:105111000280BCD2D580BAD20580B47F20125064FF
:105121002002077401B5700040F1125021FF1250A6
:105131006402509ED208D2068095125021FB125073
:1051410021FA125021F94A4B700679477A537BFFB5
:1051510020022EE570602A7E008E8275830012483F
:10516100EB60060EEE657170F0C2D5EBC0E0EAC0EF
:10517100E0E9C0E0EE1252BDD0E0F9D0E0FAD0E0B3
:10518100FB1248D2FF60AAEBC0E0EAC0E0E9C0E050
:10519100125064D0E02401F9D0E03400FAD0E0FBF1
:1051A100E5710460DCD571D980877BFF7A5279B9CA
:1051B100D202809C791080027908C206C208800858
:1051C100D2D5790A8004790AC2D5E571047002F555
:1051D10071E4FAFDFEFF125021FC7B08200113123D
:1051E1005021FD7B1030000A125021FE125021FF88
:1051F1007B20EC3382D592D55013C3E43000069F57
:10520100FFE49EFEE42001039DFDE49CFCE4CBF859
:10521100C201EC700CCFCECDCCE824F8F870F3804D
:1052210017C3EF33FFEE33FEED33FDEC33FCEB330D
:10523100FB994002FB0FD8E9EB300105F8D0E0C43F
:1052410048B201C0E00AEC4D4E4F78207B0070C29D
:10525100EAB5710040BCC0E01252BFD0F0D0E020EE
:105261000104C4C0E0C4B201C0F012504DD0F0D569
:10527100F0EB02509E124D6B513B5351B558510CFE
:105281004C51084251B94F51C14451C14951214377
:0852910051C75551AB4651AB6A
:105299004551AB4753675051102D51142E51372B9F
:1052A90051182351352053502A50D0480000512F0E
:1052B9003F3F3F00790AA2D5200314300509B910F0
:1052C900020404B9080104A2D520060250010420F1
:1052D90002689202B570005034C0E07F2030031993
:1052E9007F30A20272067205500F125316C202C213
:1052F90006C205C2087F30800F300503E9C0E012FD
:105309005064300503D0E0F9D0E0B570CC30051712
:105319007F30B9100C1250647F583004077F7880B1
:1053290003B908031250643002057F2D0250647FCF
:10533900202008F87F2B2006F322920280CF286EC6
:10534900756C6C2900D2011250213001F8C2017824
:105359007030D50108F60250D02D504349581250EB
:10536900212403B405004001E4905362931250557F
:0D537900743A125055D2037570040251B5FC
:104DC400EF4E6012EF60010EEDBB010B89828A8306
:104DD400F0A3DFFCDEFA2289F05007F709DFFCA913
:0C4DE400F022BBFEFCF309DFFCA9F0226A
:094DF000E2FB08E2FA08E2F922F4
:108CDD00EFB40A07740D128CE8740A309811A89934
:108CED00B8130CC2983098FDA899C298B811F630F7
:078CFD0099FDC299F59922CF
:00000001FF
